:020000040000FA
:06000000FE300F306A28FB
:08000800A000030EA100831209
:10001000C31D3B288B1C34288B1031181628B11CAB
:10002000342864300102031833281A2800001828E5
:1000300019281A281B281C281D281E281F2820289C
:1000400021283110B114A810031005190314AA0DAA
:10005000A90DA80DB00B342831152A08AF002908C6
:10006000AE002808AD00B11081010B11210E8300F4
:10007000A00E200E090005194328831601178312CC
:10008000B23081005E2883160113831203140B190A
:100090000310A80DA90DAA0DAB0DAC0DAC16FF30C9
:1000A0002C02031D5E28FA302B02031D5E28311539
:1000B0002A08AF002908AE002808AD008B100B11EC
:0A00C000210E8300A00E200E09009F
:0C00D400203084008001840A8030040287
:1000E000031C6C281230B0005A30C000C10001302F
:1000F000D400D500E400E500E300F100F000073093
:10010000D8008030D7001F30E6000717FA30FD0016
:100110000330EF0083160F308505203086050D3043
:1001200087058312850186018701103083168E00B2
:100130008312703083168F008312003003179900EA
:100140000313003003179A000313003097000030A8
:100150009F00003083169F008312003003179E001B
:100160000313003003179F000313C0308316810070
:1001700083123130900000309200003083169400DA
:10018000831200309400A63083169800831200304A
:1001900083169B00831290309800333083169900A9
:1001A0008312003083168C008312003083168D007A
:1001B000831210308B000D16422581018E018F01B4
:1001C0000B118B100B108C128C018D010D168B17DF
:1001D00005234323782123213119BC23311A3D21E2
:1001E000591CE822591879228F080319EB288F012E
:1001F000BB227923F421CF218F21AF210629E71BD0
:10020000EB01EB0B0629E801E901EA01E7135918B4
:10021000EB28B1191829D60BEB28B11A0A30B11EF8
:10022000C830D600B11A1F297821CC0ACC194A143B
:10023000B111B11A0A30B11EC830D600EB287821AE
:10024000BE184225EB286400C31DB113C31D08006E
:10025000311808000B1D08000B11B11031141230B9
:10026000B000051D3829B117831601138312080049
:10027000B113831601178312080031124A10CC0102
:1002800021305B02031D4A295C08CE005D08CF00C7
:10029000661773295B085C065D02031D0800773052
:1002A0005B02031D57295C087406C400732966307D
:1002B0005B02031D5E295C08CB00732955305B028D
:1002C000031D65295C08F800732944305B02031D97
:1002D0006C295C08FA00732933305B02031D732913
:1002E0005C08FB007329B116B1110A30D600080072
:1002F000591459158B138316071283128B1707167F
:1003000008005910D9101930DE00B112B111C830EF
:10031000D6008B138316071683128B170800051857
:1003200096291930C00703189B2908000A30C0021B
:10033000031CA7290800FF30C000421464304102AA
:10034000031808004210C2144317C3140800C00168
:100350004210C213C21C0800C201431308008518D2
:10036000B6291930C1070318BB2908000A30C10299
:10037000031CC7290800FF30C1004214643040024A
:1003800003180800421042154317C3100800C101AA
:100390004210C213421D0800C20143130800E303C8
:1003A000031D080065186008E518610865196208F2
:1003B00099000330E3000310E50DE519E02908007A
:1003C0001430E3000130E5001030E61AE40020307C
:1003D000661BE4000310E40D03186414640866054A
:1003E0000319E029052308008C1E0800E7174A15A9
:1003F0000717FA30FD001819CA146908E8006A08DE
:10040000E9001A08EA00E81F08006808C13C031D5B
:10041000112A69086A05C3046A096904C305AE2480
:10042000782A6808C23C031D1D2A69086A05C504AC
:100430006A096904C505B424782A6808C43C031D08
:10044000242A6908F700782A6808FC39E03C031D73
:10045000342A690868188038BB006A08E8188038B0
:10046000BA002625BE14782A6808FC39F03C031D22
:100470004E2A690868188038EC0064000D1E3E2A78
:100480008B136C0803178D0083168C130C148312C6
:100490000C080313ED008B17E616782A6808FC3960
:1004A000803C031D5D2A690868188038CE006A0800
:1004B000E8188038CF00D815782A6808FC39903CB5
:1004C000031D682A690868188038CE005816782AF3
:1004D0006808A03C031D782A69086A188038CD0096
:1004E000C310EA18C31445126A194516D816782A9B
:1004F00008005919862AD3030F305305031D08003D
:10050000D3080319892A0716D30E0800591B4F2355
:10051000591307125911D918812955185008D5189F
:100520005108551952085705031D992AFF30D30069
:100530009C2A2230D3009C2A0310D70C0318A12A2E
:1005400008008030D7000310D50DD519A82A08005F
:100550000130D5000430D819D4000830581AD4001E
:100560000310D40D03185414540858050319A82A6D
:100570004323D9140800EF0B08000330EF00061ED8
:10058000E62A05160310F00D031CD42A0130F000F2
:100590000310F10D711ED42A0130F100F00044085F
:1005A000F300C31AF317051271187308F1187208D3
:1005B00071197708F11DDF2A4B084A188038700539
:1005C000061203198516031D851208000616080079
:1005D000DA0A0319D9165916071E5912D91D012B0B
:1005E000591A012BB1155A08283CD91A0310DD0DF0
:1005F000DC0DDB0DDA01D912DE0B012B31161930BF
:10060000DE00D915591ED9110800E001E101E2010F
:10061000641F112B4830E0004E08E1004F08E20053
:100620006613E41E1A2B4730E0006C08E1006D08E9
:10063000E200E612641E222B4130E0007A08E1005D
:100640007B08E200E41D2A2B4C30E0007708E10033
:100650007808E200641D322B4530E0004A08E100D2
:100660004B08E200E41C3A2B4630E0004308E1006E
:100670004408E200641C422B5830E0005930E1008D
:100680005A30E2000800D001D101D201541C4D2B98
:10069000F730D0004308D100752BD41C542BA13067
:1006A000D0007708D100752B541D5B2BA230D000F1
:1006B0004508D100752BD41D652BC130D0004E08E4
:1006C000D1004F08D200D8110800541E6D2BC23043
:1006D000D0004E08D1005812752BD41E0800A73048
:1006E000D0004D08D100D812752B50085106D20009
:1006F0000800311F7E2BFC0303193113071F832BC6
:10070000FD0303190713031044180314B20DF0304E
:1007100032020319431307184311071C4315071925
:10072000C311071DC31587194312871D4316751C76
:100730009D2BC31E8710C31A8714FE0B0800441894
:100740009D25441C87124A1C87174A189525790A4B
:10075000F71BF707771BB02B790A77020318F7000E
:100760007808F2000310790C013E7802C3120318D6
:10077000F2000318C31608003111311B0800591884
:1007800008004A100717FA30FD00B7010430B8001E
:100790000C30370230300318B807C319B8178B1361
:1007A00020303707380703178D0083168C130C147D
:1007B00083120C080313A400A500C030A506103056
:1007C0003707380703178D0083168C130C14831218
:1007D0000C080313A300A6000230A606003037075A
:1007E000380703178D0083168C130C1483120C0822
:1007F0000313A200A7000130A7068B17B11F062C18
:1008000022090339A200A309A409A509C31D152CB7
:1008100022082D02031DA82C23082E02031DA82C3C
:1008200024082F02031D692C212C24082F02031DEC
:10083000A82C23082E02031D692C22082D02031D5B
:10084000A82C00303702031D2A2C4318080043143B
:10085000AE24080001303702031D3A2CFF30FC00A3
:100860003117441CC314441C092544184313441C69
:100870004317080002303702031D4A2CFF30FC00EA
:100880003117441CC314441C112544184313441C41
:100890004317080003303702031D512C441CC314B6
:1008A000080064000D1E522C3030370738077F399E
:1008B00003178D0083168C130C1483120C0803137A
:1008C000F7005917441CBA24FF30FC0031174418B4
:1008D0004313C31D702C25082F02031DA82C782C50
:1008E00026082E02031DA82C27082D02031DA82C64
:1008F00000303702031D812C431C08004310AE2436
:10090000080001303702031D912CFF30FC00311725
:10091000441CC310441C002544184313441C4317B3
:10092000080002303702031DA12CFF30FC003117F4
:10093000441CC310441C112544184313441C431782
:10094000080003303702031DA82C441CC310080004
:10095000B70A1C30370203180800C62B2130BB0031
:100960004308BA00262508002330BB004508BA001A
:1009700026250800771B0800431AFE2C0310790C6B
:10098000013E77020318F7000318BE2C770878029F
:100990000319DC2C0318D42C78087702C3187902C9
:1009A000C318013EFF00E32C77087802C31C7902CC
:1009B000C31C013EFF00E32C0310790C013EFF0035
:1009C000F518F707F62C0310790C013EF518013ED7
:1009D0007F02031CF62C0310790C013EF707790AFD
:1009E00077020318F7000318EF2CF62C770878022B
:1009F0004313031D4317F51843170800F62C08008E
:100A00005917C310780AF700790A77020318F7001C
:100A100008005917C3147803F700790AF71BF70782
:100A2000080059170310790C78077902031C202D50
:100A30000319202D0310790C013E7807F7000800F8
:100A40000310790C013E7802F70008000D123B08F4
:100A5000831203178D00831203133A0883120317BE
:100A60008C00831603178C130C158B138B1B352DE1
:100A700055308D00AA308D008C148B170C11831209
:100A80000313080064000D1E432DBE108B138B1B37
:100A9000462D313003178D0083168C130C148312EE
:100AA0000C080313F4008B1774108B1332300317E8
:100AB0008D0083168C130C1483120C080313F5009D
:100AC0008B178B13333003178D0083168C130C1484
:100AD00083120C080313F6008B178B1321300317B6
:100AE0008D0083168C130C1483120C080313C3009F
:100AF0008B1743138B13233003178D0083168C132E
:100B00000C1483120C080313C5008B178B133030A1
:100B100003178D0083168C130C1483120C08031317
:100B200007183030F900F90308000708803A8700F9
:100B300008000708403A870008000708203A8700A5
:100B40000800FF009D25FF0BA22D08000708023AB0
:040B50008700080012
:084000000F000000020009009E
:02400E00CC03E1
:1042000000002900FF00FF0040004200440046007B
:104210004200430040004100460047004400450082
:10422000FF00FF00FF00FF00F200F600FA00FE00B2
:10423000F000F200F400F600F800FA00FC00FE00C6
:10424000FF00FF00FF000000E500E500E500E500DD
:10425000E900E900E900E900E900E900E900E90016
:104260001800000001000000FF00FF00FF00FF0039
:104270000000010002000300040005000600070022
:104280004300420041004000470046004500440012
:104290004400450046004700400041004200430002
:1042A000F000F200F400F600F800FA00FC00FE0056
:1042B000F000F200F400F600F800FA00FC00FE0046
:1042C000ED00ED00ED00ED00ED00ED00ED00ED0086
:1042D000F100F100F100F100F100F100F100F10056
:1042E000080009000A000B000C000D000E000F0072
:1042F0001000110012001300140015001600170022
:10430000FF00FF00FF00FF000000000000000000B1
:104310000300030003000300030003000300030085
:10432000FF00FF00FF00FF00C800C800C800C80071
:10433000C800C800C800C800C800C800C800C8003D
:10434000FF00FF00FF00FF00C300F300CF00FF00ED
:104350000300C3003300F3000F00CF003F00FF0055
:10436000FF00FF00FF00FF00FF00FF00FF00FF0055
:10437000FF00FF00FF00FF00FF00FF00FF00FF0045
:10438000020002000200020002000200020002001D
:10439000000000000000000000000000000000001D
:1043A000C800C800C800C800C800C800C800C800CD
:1043B00088008800880088008800880088008800BD
:1043C0000300C3003300F3000F00CF003F00FF00E5
:1043D0000300C3003300F3000F00CF003F00FF00D5
:1043E000FF00FF00FF00FF00FF00FF00FF00FF00D5
:1043F000FF00FF00FF00FF00FF00FF00FF00FF00C5
:00000001FF
